:030000000228F6DD
:0C28F60078FFE4F6D8FD75815402293DFE
:100F2E0020000A3C2E2E2E3E004950436F6E6E65F9
:100F3E0063745245510A004950436F6E6E65637477
:100F4E00000A49504E6F41434B210A003E432C5636
:100F5E002C43432CC0E4E0EFF2E5F020D1E8EDEABB
:100F6E00EEEC49500A003E432C4D41432C253032C5
:100F7E0062583A25303262583A25303262583A2554
:100F8E00303262583A25303262583A253032625841
:100F9E002C4D414320E0E4F0E5F10A003E432C568F
:100FAE0045522C20332E3220EEF22025732025734D
:100FBE002CC2E5F0F1E8FF20495020ECEEE4F3EB13
:100FCE00FF0A004E6F762031392032303038003132
:100FDE00313A30303A3539003E432C4C442C505285
:100FEE004F473A2020202020202020202020202083
:100FFE0020202020202020202020202020202020E3
:10100E0020202020202020202020202020202020D2
:10101E0020202020202020202020202020202020C2
:10102E0020202020202020202CC4E0F2E020EFF011
:10103E00EEF8E8E2EAE828F4E0E9EB290A003E2AB5
:10104E002C312CCEF1EDEEE2EDFBE520EFE0F0E001
:10105E00ECE5F2F0FB20F1E5F2E5E2EEE3EE20E85E
:10106E00EDF2E5F0F4E5E9F1E00A003E412C413005
:10107E00312C2562752E2562752E2562752E256200
:10108E00752C495020E0E4F0E5F120E0E4E0EFF2C9
:10109E00E5F0E00A003E412C4130322C2562752EDF
:1010AE002562752E2562752E2562752C495020E01D
:1010BE00E4F0E5F120EEF1ED2E20F1E5F0E2E5F0C1
:1010CE00E00A003E412C4130332C2562752E2562FC
:1010DE00752E2562752E2562752C495020E0E4F0A0
:1010EE00E5F120F0E5E72E20F1E5F0E2E5F0E00A8B
:1010FE00003E412C4130342C2562752E2562752E12
:10110E002562752E2562752CCCE0F1EAE020F1E522
:10111E00F2E80A003E412C4130352C2562752E2511
:10112E0062752E2562752E2562752CD8EBFEE70AA8
:10113E00003E2A2C312CC4EEEF2E20EFE0F0E0EC36
:10114E00E5F2F0FB20F1E5F2E5E2EEE3EE20E8ED6C
:10115E00F2E5F0F4E5E9F1E00A003E422C533031BD
:10116E002C2562752CC6E4E0F2FC20E7E0EFF0EEF1
:10117E00F1E020F1EEE5E4E8EDE5EDE8FF20EEF23A
:10118E0020F1E5F0E2E5F0E00A003E422C53303269
:10119E002C2562752CCEE1ECE5ED20F120F1E5F089
:1011AE00E2E5F0EEEC20E1E5E720EAE2E8F2E0ED40
:1011BE00F6E8E90A003E422C5330332C2562752C9A
:1011CE00CFE5F0E5E7E0EFF3F1EA20EFF0E820EF0E
:1011DE00EEF2E5F0E520F1E2FFE7E820F120F1E59F
:1011EE00F0E2E5F0EEEC0A003E454E440A000A44F9
:1011FE00756D705820202020203030203031203066
:10120E003220303320303420303520303620303705
:10121E0020303820303920304120304220304320D9
:10122E0030442030452030460A000A3A003A200069
:10123E000A000A44756D7044202020202030302092
:10124E0030312030322030332030342030352030D1
:10125E00362030372030382030392030412030428F
:10126E0020304320304420304520304600457272F5
:10127E00206B657900526420656570726F6D0A008F
:10128E005264204D454D0A00526420436F64650A36
:10129E0000577269746520436F64650A0044656285
:1012AE0075674950204F4E0A004465627567495074
:1012BE00204F46460A004465627567557365722075
:1012CE004F6E0A00446562756755736572204F460E
:1012DE00460A0044656275674D7367204F6E0A00BB
:1012EE0044656275674D7367204F46460A00436F2B
:1012FE006E666967206C6F636B210A0057722065FA
:10130E006570726F6D0A0020536176652065657099
:10131E00726F6D210A00457272204D414321004CBF
:10132E006F61643E3E002A003C4130313D003C413D
:10133E0030323D003C4130333D003C4130343D00C5
:10134E003C4130353D003C21003C5330313D003CAA
:10135E005330323D003C5330333D003C5330353D2D
:07136E00003C5330363D0046
:06315500015100014F00D2
:10319F00C28E438910E4F58B758DB8D2ABD28E22D7
:03001B0002286652
:10286600C0E0C083C082C0D0C28E758B00758DB8A3
:10287600201D0675A61E75A6E1054FD219E5516005
:10288600020551E550D39401400215500554E55414
:10289600540F7048D225E554543F7012D2179066F3
:1028A6008BE0600A04F0E0D394B44002D21D906637
:1028B60086E0600204F0906104E0600214F0906625
:1028C6008CE0D394014003E014F0301C020552E57D
:1028D60053D394644004D21D80020553E54ED3942D
:1028E600014002154ED28ED0D0D082D083D0E032B5
:1008D000C2AFC291C290D2B5C2227D027C007F0716
:1008E0001231388F26E526646060097D017F601231
:1008F00030D3D222E4FDFC7F0B1231388F26E5265F
:1009000030E6097D04E4FF1230F7D2227D017C003D
:100910007F071231388F26E5267008FD7FFF1230E1
:10092000D3D222302203126000C288C2A8C2AA75A4
:100930008900122C9D90633EE0B4FA06A3E064CED9
:10094000607BE4F52674362526F582E43463F5836E
:10095000E4F00526E526B443EC90633E74FAF0A378
:1009600074CEF0A374CCF0906344740AF0E4A3F066
:10097000A304F0A3F090633A74FFF0A3F0A3F0E4B3
:10098000A3F0906355740AF0E4F526E5262401FFF0
:10099000E433FE74362526F582E43463F583E0FD06
:1009A0001230AF0526E526C3944340DFE4F5A77572
:1009B000A61E75A6E1907FF0F0A3F080FE9063493B
:1009C0007403F0A374CCF0E4906348F0122591C254
:1009D000B51227C7C21D122ECFD222C224C2239025
:1009E00065767408F09062B47424F0E4A3F0906328
:1009F0003EE09062B6F090633FE09062B7F09063A3
:100A000040E09062B8F0906341E09062B9F090638A
:100A100042E09062BAF0906343E09062BBF07550A0
:100A200001E4906577F0C21EC21FC220C2212022BD
:100A300018AF26FE7D031223D5E4FF1227177E0F81
:100A40007F2EE4FBFDFC1220E290668BE0600374D5
:100A500001F0E4906104F0F552906575F0F55312E1
:100A6000319F75A70775A61E75A6E1D2AFE4F553B1
:100A7000906104E070031231AF90668CE0B4011114
:100A80009080007410F0E490668CF0D222C223C2F1
:100A900024908008E0F52630E405D21E7410F0E5BD
:100AA0002630E508D2209080087420F0E52630E654
:100AB00008D21F9080087440F0E552C39403401997
:100AC000908002E4F0908001F0908000F0E5529474
:100AD000064006E4F552122ECF9080A0E07003127B
:100AE0002D1B9080B8E07003122D959080D0E0709F
:100AF00003122E0F908000E07013301E101221E9B7
:100B0000906331EFF0D394004003120026908002EE
:100B1000E07006908000E06005D21C020A6DC21CE5
:100B2000E4F552906104E06003020A6D2022129005
:100B30006578E0600C7E0F7F301222EDE4906578DE
:100B4000F0302012121E56906331EFF0D394004023
:100B500005E0FF1231DA201F03020CD6121CCF90E1
:100B60006331EFF07003020A6D906375E054BF24A7
:100B70007F7003020C3F147003020C172402600301
:100B8000020C782022077E0F7F371222ED202603E9
:100B9000020CD690634DE07006906351E060679060
:100BA0006682E0FF90634DE0B50724906683E0FE27
:100BB00090634EE0B50618906684E0FE90634FE0C7
:100BC000B5060C906685E0FE906350E06E6037904D
:100BD0006351E06F6003020CD6906683E0FF906380
:100BE00052E06F6003020CD6906684E0FF9063537E
:100BF000E06F6003020CD6906685E0FF906354E0DE
:100C00006F6003020CD6C21A9065777401F012006F
:100C10001E755001020CD690668BE060037401F0E3
:100C200090667AE0FF906377E06F6003020CD690E5
:100C3000667AE004F0E4F550906575F0020CD63069
:100C40001A03020CD6906344E07003020A6D9063AD
:100C500055740AF01231D0D21AE4F550906575F04F
:100C600090668604F0E4906679F0A3F02022677E17
:100C70000F7F451222ED805E90668BE06003740169
:100C8000F0301A52906375E020E74B906377E0FFF5
:100C9000906679E0FE6F600D906681E07007EE145B
:100CA0006F70338013906679E004F0906331E0FF59
:100CB000D394044003121FBC9060007482F0A374AC
:100CC00001F0906377E0906002F07E607F007D032A
:100CD000122A09020A6D201A03020DEEE55070680F
:100CE000122FF9EF60237E647F75906476E0240410
:100CF000FD122A09906681E07009906355E0F55075
:100D0000020A6DE4F550020A6D906686E0D3943CC9
:100D10004036906681E0703090668604F012265B63
:100D2000E4906475F0A37412F090667AE0906477B2
:100D3000F0A374FDF090610563A20190647963A251
:100D4000017F12121A1D809E12318B8F26E526B468
:100D500001159060007483F0E4A3F07E607F007D55
:100D600002122A09020A6DE526D39401401C906004
:100D7000007483F0A37401F0E52624FEA3F07E60E6
:100D80007F007D03122A09020A6DE55064016003A9
:100D9000020A6D906575E004F02022077E0F7F4FF8
:100DA0001222ED906355E0C394C85004E02432F061
:100DB000906575E0C39405400DC21AE4906577F024
:100DC00012001E020A6D7C667D82906349E0FAA3E0
:100DD000E0FB7F02122B9A7E647F75906476E0249C
:100DE00004FD122A09906355E0F550020A6DE550A2
:100DF00064016003020A6D906577E014604624FE8A
:100E00006042147003020EE124046003020A6DE4E0
:100E1000F5522026139065777404F0906575E054C0
:100E200001F0755001020A6D9080027410F0E49098
:100E30006577F090657504F07550FA90668274FFDE
:100E4000F0020A6D906682E07003020ECB9064752A
:100E50007480F09064777401F0E4A3F0A304F0A32D
:100E60007430F0A3747BF0E4F526747C2526F582BB
:100E7000E43464F583747DF0747D2526F582E434D2
:100E800064F583E4F0E5262407906476F07C667DC3
:100E900082906349E0FAA3E0FB7F02122B9A7E6402
:100EA0007F75E5262409FD122A09906681E0601B02
:100EB0001231D0D21AE4F550906575F09066860430
:100EC000F0E4906679F0A3F0020A6D302607E49012
:100ED0006577F080069065777404F07550FA020A21
:100EE0006D9080027410F0755005906575E0640196
:100EF000FFF09065777401F0EF7019906351E06036
:100F000013FCA3E0FDA3E0FEA3E0FF9066821217AE
:100F1000B0020A6D90634DE0FCA3E0FDA3E0FEA3E8
:0D0F2000E0FF9066821217B0020A6D80FE9D
:010F2D0022A1
:10002600906376E0B444047F0180027F009063759C
:10003600E0B447047E0180027E00EE5F604A906372
:100046003EE0906377F090633FE0906378F09063D2
:1000560040E0906379F0906341E090637AF09063BA
:1000660042E090637BF0906343E090637CF09063A2
:10007600767452F09062AE63A2019080A863A201EA
:100086007F06121A1D0208C6906331E0C394085019
:10009600030208CF90633EE0FF906377E06F600352
:1000A6000208CF90633FE0FF906378E06F60030241
:1000B60008CF906340E0FF906379E06F6003020829
:1000C600CF906341E0FF90637AE06F60030208CF50
:1000D600906342E0FF90637BE06F60030208CF907D
:1000E6006343E0FF90637CE06F60030208CF906398
:1000F60076E0B444159062AEE0B4FF0E63A20190C0
:1001060080A863A2017F06121A1D90668BE0600329
:100116007401F090668C7464F09063767452F0907B
:100126006375E0646D60030202537BFF7A0F795AB0
:100136001213D77BFF7A0F797490633EE0F52FA3F5
:10014600E0F530A3E0F531A3E0F532A3E0F533A303
:10015600E0F5341213D7752FFF75300F7531D17551
:1001660032FF75330F7534DD7BFF7A0F79AA1213D0
:10017600D77BFF7A0F79E61213D77BFF7A10794C7B
:100186001213D77BFF7A107979906344E0F52FA399
:10019600E0F530A3E0F531A3E0F5321213D77BFF8B
:1001A6007A1079A390634DE0F52FA3E0F530A3E034
:1001B600F531A3E0F5321213D77BFF7A1079D1908F
:1001C6006351E0F52FA3E0F530A3E0F531A3E0F5A8
:1001D600321213D77BFF7A1079FF90633AE0F52F3E
:1001E600A3E0F530A3E0F531A3E0F5321213D77B97
:1001F600FF7A117922906336E0F52FA3E0F530A35C
:10020600E0F531A3E0F5321213D77BFF7A11793F7F
:100216001213D77BFF7A117968A226E433F52F12E1
:1002260013D77BFF7A117998906681E0F52F121328
:10023600D77BFF7A1179C390668BE0F52F1213D71F
:100246001230627BFF7A1179F61213D7229063750A
:10025600E0644C60030203127E117FFCFBFDFC127E
:1002660020E290637DE0F527A3E0F528E4F52AE493
:10027600F529852882852783E0FF747F2529F58265
:10028600E43463F583EFF00529E529B410E4E527A6
:1002960090637FF0A3E528F07E127F387C637D7F34
:1002A6007B021220E2E4F529852882852783E0FF78
:1002B600747F2529F582E43463F583EFF00528E59C
:1002C60028700205270529E529B410DC7E127F3B3C
:1002D6007C637D7F7B101220E2E4F52985288285E8
:1002E6002783E0FF747F2529F582E43463F583EFE5
:1002F600F00529E529B410E4052AE52AC39410502F
:10030600030202757E127F3E1222ED22906375E093
:10031600646C60030203B3F52B7E127F40FBFDFC89
:100326001220E2E4F52AE4F529A82BE6FF747F25DE
:1003360029F582E43463F583EFF00529E529B41045
:10034600E8E490637FF0A3E52BF07E127F387C63B0
:100356007D7F7B021220E2E4F529A82BE6FF747F5D
:100366002529F582E43463F583EFF0052B0529E5AD
:1003760029B410E67E127F3B7C637D7F7B101220C2
:10038600E2E4F529A82BE6FF747F2529F582E434FB
:1003960063F583EFF00529E529B410E8052AE52A77
:1003A600C3940840817E127F3E1222ED229063752F
:1003B600E0644B7061F52974672529F582E434639E
:1003C600F583E0603274672529F582E43463F583AA
:1003D600E0F4602374672529F582E43463F583E04D
:1003E600FF747D2529F582E43463F583E0B50710B3
:1003F6000529E529B408C09061047432F00208C6E4
:100406009063757421F03022030208C67E127F7B4A
:100416001222ED0208C6906375E0B4521A20220734
:100426007E127F831222ED9063757472F07E637F75
:10043600757D0812298222906375E0644970452013
:1004460022077E127F8E1222ED90637DE0F527A3B0
:10045600E0F528E4F529852882852783E0FF747F67
:100466002529F582E43463F583EFF00528E5287045
:100476000205270529E529B480DC7E637F757D8A20
:1004860012298222906375E0644370462022077E1B
:10049600127F961222ED90637DE0F527A3E0F52802
:1004A600E4F529852882852783E493FF747F25292F
:1004B600F582E43463F583EFF00528E5287002053C
:1004C600270529E529B480DB7E637F757D8A12299D
:1004D6008222906375E0645A70532022077E127F51
:1004E6009F1222ED90637DE0F527A3E0F5287C635B
:1004F6007D7F7B80AF28AE2712302EE4F529852834
:1005060082852783E493FF747F2529F582E434638B
:10051600F583EFF00528E528700205270529E5296A
:10052600B480DB7E637F757D8A1229822290637593
:10053600E0644460030205C490637DE0FF64447098
:10054600030208C6EFB4310CC2227E127FAB122220
:10055600ED0208C690637DE0B4300CD2227E127F95
:10056600B71222ED0208C690637DE0B4320CD223A6
:100576007E127FC41222ED0208C690637DE0B4337A
:100586000CC2237E127FD21222ED0208C690637D32
:10059600E0B4340CD2247E127FE11222ED0208C6AA
:1005A60090637DE0B4350CC2247E127FEE1222EDFC
:1005B6000208C690637DE0FF1231D90208C6906139
:1005C60004E070132022077E127FFC1222ED906356
:1005D600757421F00208C69061047432F090637558
:1005E600E0FFB45104C2AF80FEEF6457704520228D
:1005F600077E137F0A1222ED90637EE0906331F04E
:10060600E4F529906331E0FFE529C39F4003020822
:10061600C6747F2529F582E43463F583E0FF906391
:100626007DE0252924ADF582E43461F583EFF005FC
:100636002980D0906375E0645360030206E72022A8
:10064600077E137F151222ED90633EE0FF9061B6A0
:10065600E06F703C90633FE0FF9061B7E06F7030F1
:10066600906340E0FF9061B8E0B50724906341E0F5
:10067600FF9061B9E0B50718906342E0FF9061BA58
:10068600E0B5070C906343E0FF9061BBE06F601636
:100696009063757421F03022030208C67E137F240E
:1006A6001222ED0208C6E4F529E4F553AF29FE74DB
:1006B600AD2529F582E43461F583E0FD1230AF05FE
:1006C60029E529C394FE40E1C2AFE4907FF0F0A390
:1006D600F0907FFD74AAF0A374FFF0A37455F08028
:1006E600FE906375E0644F704C90637DE0F527A340
:1006F600E0F528E5284527700A2022077E137F2D7E
:100706001222ED2022077E137F341222EDE4F52912
:10071600747F2529F582E43463F583E08528828594
:100726002783F00528E528700205270529E529B461
:1007360080DE0208C6906375E0FFB4452190637DB4
:10074600E0FDA3E0907FF0CDF0A3EDF0C2AF907F87
:10075600FD74AAF0A374FFF0A37455F080FEEF6455
:100766006560030208CF90637DE0FFA3E0907FF011
:10077600CFF0A3EFF0E4F527F528D3907FF1E095CD
:1007860028907FF0E095274020E4F5532528FFE5E3
:10079600273401FE852882852783E0FD1230AF05C8
:1007A60028E5287002052780D17E137F36122A900D
:1007B600EF4E6020120003906344EFF012000390A6
:1007C6006345EFF0120003906346EFF012000390CA
:1007D6006347EFF07E137F3C122A90EF4E602012A3
:1007E600000390634DEFF012000390634EEFF0129A
:1007F600000390634FEFF0120003906350EFF07E1A
:10080600137F42122A90EF4E60201200039063512C
:10081600EFF0120003906352EFF01200039063535F
:10082600EFF0120003906354EFF07E137F48122A14
:1008360090EF4E602012000390633AEFF01200032F
:1008460090633BEFF012000390633CEFF01200035D
:1008560090633DEFF07E137F4E122A90EF4E60209C
:10086600120003906336EFF0120003906337EFF047
:10087600120003906338EFF0120003906339EFF033
:10088600E4F529E4F553E5292401FFE433FE743643
:100896002529F582E43463F583E0FD1230AF05299E
:1008A600E529C3944340DCC2AFE4907FF0F0A3F0A7
:1008B600907FFD74AAF0A374FFF0A37455F080FE38
:0908C6007E637F757D0812298212
:0108CF002206
:102FC100AE07EEC39430400BEED394395005EE2496
:102FD100D0FF22EEC39461400BEED394665005EE10
:102FE10024A9FF22EEC39441400BEED39446500531
:082FF100EE24C9FF22AF062205
:103171009062ADE004F070069062ACE004F0906201
:0A318100ACE0FEA3E0FF12311B22B8
:10000300123171122FC1EFC454F0FEC006123171C8
:08001300122FC1D0E02FFF22E3
:102E7200E49069C8F01231719069C9EFF0C39430DF
:102E82004018E0FFD3943950119069C8E02405F549
:102E920082E43461F583EFF080119069C8E0240583
:102EA200F582E43461F583E4F0800C9069C8E004B3
:102EB200F0E0D3940840BE752A00752B00752C00F3
:0C2EC200E4F52D7B017A617905121B2BD1
:012ECE0022E1
:042A90008E2C8F2DCC
:102A94009062ACE4F0A374FFF0123171EF606EF455
:102AA400606B852D82852C83E493B507EC752E012C
:102AB400E52D252EF582E4352CF583E493602590ED
:102AC40062ADE0252EFF9062ACE03400FE12311BB3
:102AD400E52D252EF582E4352CF583E493B5070422
:102AE400052E80CCE52D252EF582E4352CF583E4E6
:102AF4009370A6E52E24FFFFE434FFFE9062ADE060
:102B04002FF09062ACE03EF07E007F0122E4FEFFF5
:012B1400229E
:102591007E137F54122A90EF4E70037F01227E1327
:1025A1007F57122A90EF4E600C123171EF24D02424
:1025B100FF92268002D2267E137F5D122A90EF4E73
:1025C100600C123171EF24D0906681F08005E490A7
:1025D1006681F07E137F63122A90EF4E600C1231F8
:1025E10071EF24D090668BF08005E490668BF07ECD
:1025F100137F69122A90EF4E600C123171EF24D0D3
:1026010024FF92188002C21890633E63A201906673
:102611007B63A2017F06121A1D30183B7E137F6F68
:10262100122A90EF4E603012000390667BEFF01299
:10263100000390667CEFF012000390667DEFF012CC
:10264100000390667EEFF012000390667FEFF012B8
:0A2651000003906680EFF07F002286
:102F7A00906576E0C3947C503D906576E0FE04F05F
:102F8A0074B42EF582E43462F583EFF0BF0A279019
:102F9A006576E0FF04F074B42FF582E43462F583B9
:102FAA00E4F0906576E0FF122B159065767408F0D0
:072FBA009062B5E004F02273
:102ECF009080007480F090633663A201F583F582E1
:102EDF0063A2017F08121A1D90633E63A2019080C6
:102EEF008863A2017F0A121A1D908092E4F0A374E6
:102EFF0032F0A37401F0906348E0FF9080B1F0903E
:102F0F0080E1EFF09080957455F0A3F090800074FD
:092F1F0001F090800974F0F02229
:102D1B00908009E04410F09080A0E0706C9080A14E
:102D2B007482F09080A874FFF0A3F0A3F0A3F07F5F
:102D3B00039080AEEFF07FCBA3EFF07F039080ACDE
:102D4B00EFF0A374CBF09080007402F09069BA128C
:102D5B0017BC000000009069BAE0908040F09069C9
:102D6B00BBE0908041F09069BCE0908042F09069AC
:102D7B00BDE0908043F0A3E4F0A3F0A3F0A3F090A8
:092D8B008018F0A3F0A3F0A3F0FE
:012D9400221C
:102E0F00908009E04440F09080D17482F090634943
:102E1F00E0FF9080DEF090634AE0FF9080DFF0905B
:102E2F0080027402F09069BE1217BC00000000907F
:102E3F0069BEE0908058F09069BFE0908059F090A3
:102E4F0069C0E090805AF09069C1E090805BF0A378
:102E5F00E4F0A3F0A3F0A3F0908030F0A3F0A3F080
:022E6F00A3F0CE
:012E7100223E
:102D9500908009E04420F09080B8E0706C9080B994
:102DA5007482F07F039080C6EFF07FCDA3EFF07FB4
:102DB500039080C4EFF0A374CDF09080C074FFF051
:102DC500A3F0A3F0A3F09080017402F09069C21201
:102DD50017BC000000009069C2E090804CF090693B
:102DE500C3E090804DF09069C4E090804EF090690A
:102DF500C5E090804FF0A3E4F0A3F0A3F0A3F0901A
:092E05008024F0A3F0A3F0A3F077
:012E0E0022A1
:102B9A008C278D28A907EAFDE975F018A424ACFF53
:102BAA00E5F034808F82F583EDF0EBFDE975F018DE
:102BBA00A4FFAEF024ACFBEE34808B82F583A3ED48
:102BCA00F08528828C83E0FDEF24A8FFEE3480FE96
:102BDA008F82F583EDF08528828C83A3E08F828E25
:102BEA0083A3F0852882852783A3A3E0FDE975F0F6
:102BFA0018A424A8FFE5F03480FE8F82F583A3A3EE
:102C0A00EDF08528828C83A3A3A3E08F828E83A311
:042C1A00A3A3F0225E
:062982008D2CAB07AA0634
:10298800908000E030E5079065787401F022906946
:10299800BAE0FCA3E0FDA3E0FEA3E0F5308E2F8DA6
:1029A8002E8C2DAE02AF038E838F8263A201E52F9A
:1029B800540744C0F58385308263A201AF2C121AF4
:1029C8008FE4FCFDFEE530252CF530EE352FF52F94
:1029D800ED352EF52EEC352DF52D908040E52DF0BA
:1029E800A3E52EF0A3E52FF0A3E530F09080007466
:1029F80020F0AF30AE2FAD2EAC2D9069BA1217B0C3
:012A080022AB
:062A09008D27AB07AA06B1
:102A0F00908002E030E5079065787403F0229069BA
:102A1F00BEE0FCA3E0FDA3E0FEA3E0F52B8E2A8D24
:102A2F00298C28AE02AF038E838F8263A201E52A21
:102A3F00540744D0F583852B8263A201AF27121A66
:102A4F008FE4FCFDFEE52B2527F52BEE352AF52A25
:102A5F00ED3529F529EC3528F528908058E528F033
:102A6F00A3E529F0A3E52AF0A3E52BF090800274EB
:102A7F0020F0AF2BAE2AAD29AC289069BE1217B04B
:012A8F002224
:022717008F270A
:10271900908001E030E5099065787402F07F00222D
:102729009069C2E0FCA3E0FDA3E0FEA3E0F52B8ED7
:102739002A8D298C2890667B63A201E52A540744D7
:10274900C8F583852B8263A2017F06121AA5E52BA2
:102759002406F52BE4352AF52AE43529F529E4354B
:1027690028F52890657963A201E52A540744C8F53C
:1027790083852B8263A201AF27121AA5E4FCFDFE13
:10278900E52B2527F52BEE352AF52AED3529F529EF
:10279900EC3528F52890804CE528F0A3E529F0A32D
:1027A900E52AF0A3E52BF09080017420F0AF2BAE61
:0D27B9002AAD29AC289069C21217B0AF27D5
:0127C60022F0
:1021E9009081E0E0F527052705270527052705271D
:1021F90005270527052705270527908010E0F52ADB
:10220900A3E0F52BA3E0F52CA3E0F52D9081E1E007
:10221900F527052705270527052705270527052765
:10222900052705270527908014E0F52EA3E0F52F53
:10223900A3E0F530A3E0F531E530B52C08E531B57B
:102249002D037F0022E4F527E530540744E0F583A8
:1022590085318263A20190637563A2017F08121A16
:10226900D590637763A2019062AE63A2017F0612E3
:102279001A1D906375E0F528A3E0F529E4F5279088
:102289006375E0702AA3E024F8F527E53054074484
:10229900E0F58385318274082582F582E43583F57A
:1022A9008363A20190637563A201AF27121AD5AEA9
:1022B90028E4FCFDE5312529F531E5303EF530ED21
:1022C900352FF52FEC352EF52E908014E52EF0A341
:1022D900E52FF0A3E530F0A3E531F09080007440DC
:0322E900F0AF272C
:0122EC0022CF
:101CCF009081E6E0F5270527052705270527052736
:101CDF0005270527052705270527908028E0F52AE2
:101CEF00A3E0F52BA3E0F52CA3E0F52D9081E7E021
:101CFF00F527052705270527052705270527052785
:101D0F0005270527052790802CE0F52EA3E0F52F5A
:101D1F00A3E0F530A3E0F531E4F527E530B52C0A63
:101D2F00E531B52D05C21F021E3BE530540744F0C7
:101D3F00F58385318263A20190637563A2017F08E9
:101D4F00121AD5906375E0F528A3E0F529E529452A
:101D5F002870099080027410F07F0022906682E054
:101D6F00FFF46030906377E06F6003021E029066AD
:101D7F0083E0FF906378E06F7079906684E0FF9066
:101D8F006379E06F706D906685E0FF90637AE06F26
:101D9F006031805F906377E0906682F0906378E0C7
:101DAF00906683F0906379E0906684F090637AE0B8
:101DBF00906685F090637BE0FFA3E0906349CFF0DE
:101DCF00A3EFF0906375E0702AA3E024F8F527E500
:101DDF0030540744F0F58385318274082582F582EB
:101DEF00E43583F58363A20190637563A201AF2786
:101DFF00121AD5AE28E4FCFDE5312529F531E53081
:101E0F003EF530ED352FF52FEC352EF52EAF2DAEEF
:101E1F002CAD2BAC2AAB31AA30A92FA82ED3121779
:101E2F009F40099080027410F07F002290802CE573
:101E3F002EF0A3E52FF0A3E530F0A3E531F090806D
:061E4F00027440F0AF2711
:011E5500226A
:101E56009081E3E0F52705270527052705270527B0
:101E66000527052705270527052790801CE0F52A65
:101E7600A3E0F52BA3E0F52CA3E0F52D9081E4E09B
:101E8600F5270527052705270527052705270527FC
:101E9600052705270527908020E0F52EA3E0F52FDE
:101EA600A3E0F530A3E0F531E4F527E530B52C0ADB
:101EB600E531B52D05C220021FA1E530540744E8DF
:101EC600F58385318263A20190600463A2017F0ECF
:101ED600121AEB906004E0F528A3E0F52990600C57
:101EE600E0FFF4604590667BE0FEEF6E706EA3E067
:101EF600FF90600DE06F706490667DE0FF90600E6D
:101F0600E06F705890667EE0FF90600FE06F704C57
:101F160090667FE0FF906010E06F7040906680E012
:101F2600FF906011E06F60048032D2D9906004E0C7
:101F3600702AA3E024F2F527E530540744E8F58338
:101F4600853182740E2582F582E43583F58363A29A
:101F56000190600463A201AF27121AEBAE28E4FCDD
:101F6600FDE5312529F531E5303EF530ED352FF526
:101F76002FEC352EF52EAF2DAE2CAD2BAC2AAB317A
:101F8600AA30A92FA82ED312179F5006E529452857
:101F960070099080017410F07F0022908020E52E59
:101FA600F0A3E52FF0A3E530F0A3E531F090800132
:051FB6007440F0AF27AC
:011FBB002203
:0422ED008E2C8F2D77
:1022F100908000E030E5079065787401F0229069E4
:10230100BAE0FCA3E0FDA3E0FEA3E0F5338E328D3D
:10231100318C30E533FFE5325407FEE42FF52FEE23
:1023210034C0F52E852F82F5837423F0052FE52F18
:102331007002052E532EC7F582852E83740AF0058F
:102341002FE52F7002052E532EC790633E63A20125
:10235100852E83852F8263A2017F06121A8F740650
:10236100252FF52FE4352EF52E852C83852D8263BF
:10237100A201852E83852F8263A201121A73E4FCC8
:10238100FDFE9069BAE0F8A3E0F9A3E0FAA3E02F1B
:10239100FFEE3AFEED39FDEC38FCEF2408FFE43E98
:1023A100FEE43DFDE43CFC9069BA1217B09069BAB5
:1023B100E0908040F09069BBE0908041F09069BC72
:1023C100E0908042F09069BDE0908043F090800001
:0323D1007420F085
:0123D40022E6
:0A20E2008E2C8F2D8C2E8D2F8B304D
:1020EC00908000E030E5079065787401F0229069EB
:1020FC00BAE0FCA3E0FDA3E0FEA3E0F5368E358D3F
:10210C00348C33E536FFE5355407FEE42FF532EE1B
:10211C0034C0F531853282F5837423F00532E53213
:10212C00700205315331C7F582853183740AF0058D
:10213C0032E532700205315331C790633E63A20120
:10214C0085318385328263A2017F06121A8F740651
:10215C002532F532E43531F531852C83852D8263BA
:10216C00A20185318385328263A201121A738F37E3
:10217C00EF2532F532E43531F531E5306017852E37
:10218C0083852F8263A20185318385328263A2010C
:10219C00AF30121A8FE53724082530F530FFE4FCF8
:1021AC00FDFEE5362FF536EE3535F535ED3534F5E6
:1021BC0034EC3533F533908040E533F0A3E534F05F
:1021CC00A3E535F0A3E536F09080007420F0AF362F
:0C21DC00AE35AD34AC339069BA1217B0C8
:0121E80022D4
:0624B6008E458F468D47A4
:1024BC00908000E030E5079065787401F022906917
:1024CC00BAE0FCA3E0FDA3E0FEA3E0F54D8E4C8D3D
:1024DC004B8C4AE54DFFE54C5407FEE42FF549EED5
:1024EC0034C0F548854982F5837423F00549E549E4
:1024FC00700205485348C7F582854883EBF00549BF
:10250C00E549700205485348C790633E63A20185B4
:10251C00488385498263A2017F06121A8F740625AF
:10252C0049F549E43548F54885458385468263A2DB
:10253C000185488385498263A201AF47121A8F74C3
:10254C00082547F547FFE4FCFDFEE54D2FF54DEE64
:10255C00354CF54CED354BF54BEC354AF54A908046
:10256C0040E54AF0A3E54BF0A3E54CF0A3E54DF0B4
:10257C009080007420F0AF4DAE4CAD4BAC4A9069DE
:04258C00BA1217B0B8
:012590002228
:022B15008F40EF
:102B1700908000E030E5079065787401F0229069B5
:102B2700BAE0FCA3E0FDA3E0FEA3E0F5448E438DED
:102B3700428C41E544FFE5435407FEE42FFFEE34A2
:102B4700C09062B463A201F5838F8263A201AF4094
:102B5700121A8FE4FCFDFEE5442540F544EE3543AB
:102B6700F543ED3542F542EC3541F541908040E5BE
:102B770041F0A3E542F0A3E543F0A3E544F09080DC
:102B8700007420F0AF44AE43AD42AC419069BA1235
:022B970017B075
:012B99002219
:0623D5008E278F28AB05E6
:1023DB00908000E030E5079065787401F0229069F9
:1023EB00BAE0FCA3E0FDA3E0FEA3E0F52E8E2D8D5D
:1023FB002C8C2BE52EFFE52D5407FEE42FF52AEE52
:10240B0034C0F529852A82F5837423F0052AE52A41
:10241B00700205295329C7F582852983EBF0052A1C
:10242B00E52A7002052990633E63A2018529838505
:10243B002A8263A2017F06121A8F7406252AF52AB7
:10244B00E43529F5295329C7E527852A8285298370
:10245B00F0052AE52A700205295329C7F58285293B
:10246B0083E528F0052AE52A700205295329C7E5DB
:10247B002E240AF52EE4352DF52DE4352CF52CE420
:10248B00352BF52B908040E52BF0A3E52CF0A3E545
:10249B002DF0A3E52EF09080007420F0AF2EAE2D22
:0A24AB00AD2CAC2B9069BA1217B0EB
:0124B5002204
:0A31BB00E4FEEEC39F50030E80F8FF
:0131C50022E7
:10311B00A2AF9227C2AF438E2075D2028F828E83CD
:0C312B00E0FFE4F5D2538EDFA22792AF44
:013137002275
:1030AF00E5D220E0FBA2AF9227C2AF43D2028F82BC
:1030BF008E83EDF075D25063D250A22792AFE5D236
:0330CF0020E0FB03
:0130D20022DB
:102C9D00E4FDED2401FFE433FE12311B74362DF5F6
:102CAD0082E43463F583EFF00DBD3FE6E4FDED24E2
:102CBD007FFFE433FE12311B742D2DF582E4346158
:102CCD00F583EFF0742D2DF582E43461F583E0701A
:102CDD001B742D2DF582E43461F5837420F0742E70
:102CED002DF582E43461F583E4F080040DBD80BEE2
:102CFD00E49061ACF0FDEDFF7E0012311B74AD2D43
:0D2D0D00F582E43461F583EFF00DBDFEE9C1
:012D1A002296
:02302E008B2CE9
:10303000A2AF9227C2AF85A22D53A2FE8E838F82AC
:1030400005A28C838D827409121B19E52C53A2FEF4
:1030500043A220121B1B53A2DF852DA2A22792AFF1
:01306000FF70
:01306100224C
:10313800A2AF9227C2AF8C838D82EF121B1943A2D4
:0C31480020121B1B53A2DFA22792AFFF36
:013154002258
:0230D3008F2745
:1030D500A2AF9227C2AFE4F5838D827406121B1945
:1030E500E52743A220121B1B53A2DFA22792AF7F25
:0130F50001D9
:0130F60022B7
:0230F7008F2721
:1030F900A2AF9227C2AFE4F5838D82740A121B191D
:10310900E52743A220121B1B53A2DFA22792AF7F00
:0131190001B4
:01311A002292
:10194200A907E7FFA805EF93C3966008403B74FC24
:101952002FFF80F00F08EF93C3966008402B74FBB3
:101962002FFF80E00F08EF93C3966008401B74FAC4
:101972002FFF80D00F08EF93D3966008400B74F9C5
:101982002FFF80C01F1F1F1F1FEF54FEF80303F716
:10199200E893FC08E893FD08E893FE08E893FF2229
:1019A20009E993C39D6008402974FB29F980F10974
:1019B200E993C39E6008401A74FA29F980E209E9A2
:1019C20093D39F6008400B74F929F980D319191930
:1019D2001919E9C313C313FF22740093F8ECC398D7
:1019E2004024701F740193F8EDC398401970147469
:0E19F2000293F8EEC398400E7009740393F848
:101A0000EFC39840037F00227F0122EDF8E6F00843
:101A1000A3DFFA22EDF8E0F608A3DFFA22E0A363E1
:101A2000A201F0A363A201DFF475A2002263A20168
:101A3000F0A363A20122E0A363A201F0A363A201C9
:101A4000E0A363A201F0A363A201E463A201F0A3F7
:101A500063A201DFE175A20022E0A363A2016DFE93
:101A6000936CFDEE058393FC158363A201DFEA7599
:101A7000A200227F00E493A363A201F00F600CA3F5
:101A8000E583C2E3F58363A20180EA75A20022E048
:101A9000A363A201F0A3E583C2E3F58363A201DFA0
:101AA000EE75A20022E0A363A201F0A3E583C2E4E5
:101AB000D2E3F58363A201DFEC75A20022E0A36309
:101AC000A201F0A3E58344F8C2E5F58363A201DF38
:101AD000EC75A20022E583C2E3F583E0A363A201D3
:101AE000F0A363A201DFEE75A20022E583C2E4D277
:0A1AF000E3F583E0A363A201F0A375
:101AFA0063A201DFEC75A20022E58344F8F583E0D6
:101B0A00A363A201F0A363A201DFEE75A20022F98A
:101B1A0022C002C004C00612FFF0D006D004D002D0
:011B2A002298
:102C1E003E2A2C312CC2FBE2EEE420E4E0EDEDFB8B
:102C2E00F520EDE020F2E0E1EBEE20D0D3C1C8CDEF
:102C3E002E0A003E532C4730332C256C752CC7E0E2
:102C4E00E4E5F0E6EAE020F1F2E0F0F2E020EFE574
:102C5E00F0E5E4E0F7E828ECF1290A003C473033D0
:102C6E003D000A496E707574205061636B65743A4D
:102C7E0020000AC1F3F4E5F020E7E0EDFFF22100B9
:0F2C8E000A53656E64205061636B65743A2000D1
:10315B0052668D000000000000000000000000001F
:05316B0000000000005F
:0131D90022D3
:03002300022F2881
:102F2800C0E0C083C082C0D075D018309802C29863
:102F380030993430032F9066A1E0FFE510C39F401D
:102F480011C203D213C290200B02D215C20BD29623
:102F58008013AF10051074AF2FF582E43468F58341
:102F6800E0F511F599C299D2AFD0D0D082D083D0F4
:022F7800E03245
:103062007BFF7A2C791E1213D77BFF7A2C79419041
:1030720068AEE075F00AA4FFAEF0E48F328E31F54F
:0730820030F52F1213D722D5
:103089007E2C7F6A122A90EF4E6013122E72E47B17
:103099000AFAF9F812170D9068AEEFF08005E4907E
:0630A90068AEF07F00227A
:1027C700C203C215C208C202C20FE4F5109066A187
:1027D700F0F50EF551C200D297D296750CFF9067AF
:1027E700ADF075080CC206C21490669F7409F0A379
:1027F700F0750F05C209C204C201C212C210D20C81
:10280700E4F50AF509D2139069B474FFF0A374B81C
:10281700F0C20AC205C211E4F50D123089E49067CF
:10282700A2F0C2ADF5C9D2CDD2CCC2C9C2CAF5CDCC
:10283700F5CC9069B4E0F5CBA3E0F5CA85CBCD859F
:10284700CACCE4F598D29E438740C29FC2ACC298D7
:0F285700C29975B81075B710D2CAD29CD2AC22F4
:0131DA0022D2
:10265B00E4FF9066A0E0FE7D000FED2405F582E41B
:10266B003461F583EEF00F74052401F582E43461D7
:10267B00F583E4F07C667D92FEED1DAA0470011CCF
:10268B00F5828A83E0FBAA070F74052AF582E434EE
:10269B0061F583EBF00EBE04E07C667D96E4FEED07
:1026AB001DAA0470011CF5828A83E0FBAA070F7434
:1026BB00052AF582E43461F583EBF00EBE04E07C71
:1026CB00667D9AE4FEED1DAA0470011CF5828A83D7
:1026DB00E0FBAA070F74052AF582E43461F583EB5E
:1026EB00F00EBE04E07C667D9EE4FEED1DAA047038
:1026FB00011CF5828A83E0FBAA070F74052AF58279
:0B270B00E43461F583EBF00EBE04E047
:0127160022A0
:0A31C600C2992099FDD299D29022FF
:0931D000D2CAD29CD2ACC2082282
:021FBC00AB0771
:101FBE0030240F7E2C7F707C637D79EB24FCFB122A
:101FCE0020E23003122024030220E17E2C7F80E4E5
:101FDE00FBFDFC1220E222906378E090669FF09069
:101FEE006379E09069AFF090637AE09069B0F09019
:101FFE00637BE09069B1F0642E60030220E190688B
:10200E00AF7410F090637AE09068B0F0146028041A
:10201E00704B75270690637DE09068B1F090637EFB
:10202E00E09068B2F0906380E09068B3F0906381C6
:10203E00E09068B4F0804C752702747B2527F582FA
:10204E00E43463F583E0FF74AF2527F582E434684A
:10205E00F583EFF00527E527B407DF802675270205
:10206E00747B2527F582E43463F583E0FF74AF2596
:10207E0027F582E43468F583EFF00527E527B408E9
:10208E00DF8000AF27052774AF2FF582E43468F5A3
:10209E00837410F0AF27052774AF2FF582E43468F0
:1020AE00F58374FEF09066A1E527F0E4F510D203F7
:1020BE00C296C2151231C69068AEE004F5093024FE
:1020CE00127F141231BB7E2C7F8E7C687DAFAB27C6
:0320DE001220E2EB
:0120E10022DC
:102FF90030162FE4906475F0A37403F090667AE0BC
:10300900906477F090669FE0906478F09069AF6380
:10301900A20190647963A2017F03121A1DC2167F6F
:0530290001227F0022DE
:05001E00C2AEC2AC22DD
:0C31AF00301908C219E509600215092258
:10318B0030150EE50960037F0022C215D2167F01B0
:04319B00227F00226D
:102902000208D0E493A3F8E493A34003F68001F213
:1029120008DFF48029E493A3F85407240CC8C333D6
:10292200C4540F4420C8834004F456800146F6DFA5
:10293200E4800B0102040810204080903155E47EAF
:10294200019360BCA3FF543F30E509541FFEE4939A
:10295200A360010ECF54C025E060A840B8E493A361
:10296200FAE493A3F8E493A3C8C582C8CAC583CA8C
:10297200F0A3C8C582C8CAC583CADFE9DEE780BE44
:01317000005E
:1016D10075F008758200EF2FFFEE33FECD33CDCCD0
:1016E10033CCC58233C5829BED9AEC99E582984053
:1016F1000CF582EE9BFEED9AFDEC99FC0FD5F0D630
:10170100E4CEFBE4CDFAE4CCF9A88222B800C1B959
:101711000059BA002DEC8BF084CFCECDFCE5F0CB97
:10172100F97818EF2FFFEE33FEED33FDEC33FCEBD0
:1017310033FB10D703994004EB99FB0FD8E5E4F98B
:10174100FA227818EF2FFFEE33FEED33FDEC33FC78
:10175100C933C910D7059BE99A4007EC9BFCE99A6C
:10176100F90FD8E0E4C9FAE4CCFB2275F010EF2FB1
:10177100FFEE33FEED33FDCC33CCC833C810D707B1
:101781009BEC9AE899400AED9BFDEC9AFCE899F8EC
:0E1791000FD5F0DAE4CDFBE4CCFAE4C8F9227F
:10179F00EB9FF5F0EA9E42F0E99D42F0E89C45F0A0
:0117AF002217
:0C17B000ECF0A3EDF0A3EEF0A3EFF022AC
:1017BC00A8828583F0D083D0821217D31217D3124C
:1017CC0017D31217D3E473E493A3C583C5F0C58371
:1017DC00C8C582C8F0A3C583C5F0C583C8C582C877
:0117EC0022DA
:10137500E53B242FF8E6053B22782C302E02782F0A
:10138500E475F0011218A20217ED2027EB7F2ED28B
:10139500278018EF540F2490D43440D4FF302B0B02
:1013A500EF24BFB41A0050032461FFE53C60021529
:1013B5003C053FE53F7002053E302E0D782CE47567
:1013C500F0011218A2EF021833022F7A7403D22EFD
:1013D5008003E4C22EF53B8B2C8A2D892EE4F53C47
:1013E500F53EF53FE53C60077F201213B080F575AB
:1013F5003DFFC228C227C229C22AC22CC22DC22F34
:1014050012137EFF700D302E057F001213C1AF3F02
:10141500AE3E22B4255FC2D5C22B12137EFF24D067
:10142500B40A00501A75F00A783C30D50508B6FFA5
:101435000106C6A426F620D5047002D22A80D92436
:10144500CFB41A00EF5004C2E5D22B0215C1D22841
:1014550080C6D22780C0D22980BCD2D580BAD22CF2
:1014650080B47F201213B02029077401B53C0040D9
:10147500F1121375FF1213B00213E9D22FD22D808A
:1014850095121375FB121375FA121375F94A4B7001
:101495000679927A167BFF20292EE53C602A7E008C
:1014A5008E8275830012180660060EEE653D70F09B
:1014B500C2D5EBC0E0EAC0E0E9C0E0EE121608D004
:1014C500E0F9D0E0FAD0E0FB1217EDFF60AAEBC01F
:1014D500E0EAC0E0E9C0E01213B0D0E02401F9D0A1
:1014E500E03400FAD0E0FBE53D0460DCD53DD98071
:1014F500877BFF7A167904D229809C79108002793E
:1015050008C22DC22F8008D2D5790A8004790AC273
:10151500D5E53D047002F53DE4FAFDFEFF121375B5
:10152500FC7B08202813121375FD7B1030270A1247
:101535001375FE121375FF7B20EC3382D592D550BF
:1015450013C3E43027069FFFE49EFEE42028039D95
:10155500FDE49CFCE4CBF8C228EC700CCFCECDCCDE
:10156500E824F8F870F38017C3EF33FFEE33FEED90
:1015750033FDEC33FCEB33FB994002FB0FD8E9EB71
:10158500302805F8D0E0C448B228C0E00AEC4D4E3A
:101595004F78207B0070C2EAB53D0040BCC0E01228
:1015A500160AD0F0D0E0202804C4C0E0C4B228C098
:1015B500F0121399D0F0D5F0EB0213E912190114CA
:1015C500865315005814574C14534215044F150CE7
:0F15D50044150C49146C4315125514F64614F6C0
:1015E4004514F64716B250145B2D145F2E14822B4B
:1015F400146323148020169B2A141B480000147AB9
:101604003F3F3F00790AA2D5202A14302C09B91093
:10161400020404B9080104A2D5202D0250010420BB
:1016240029689229B53C005034C0E07F20302A1943
:101634007F30A229722D722C500F121661C229C25A
:101644002DC22CC22F7F30800F302C03E9C0E01252
:1016540013B0302C03D0E0F9D0E0B53CCC302C17DB
:101664007F30B9100C1213B07F58302B077F78806D
:1016740003B908031213B03029057F2D0213B07F7C
:1016840020202FF87F2B202DF322922980CF286E43
:10169400756C6C2900D2281213753028F8C228788A
:1016A4003C30D50108F602141B2D5043495812133F
:1016B400752403B405004001E49016AD931213A100
:0D16C400743A1213A1D22A753C04021500DD
:101B2B008B278A288929E4F533F532F531F530F521
:101B3B002EF52FE52B452C452A6012EBC0E0EAC0B1
:101B4B00E0E9C0E0AB2AAA2BA92C1218B2AB2705EF
:101B5B0029E529AA287002052814F91217EDF53486
:101B6B00C394094007E534D3940D40E1E534642078
:101B7B0060DBE534B42D05432F038016E534B42B1D
:101B8B0005432F01800C74FF2529F52974FF352897
:101B9B00F528E52D60046410703FAB27AA28A9290E
:101BAB001217ED64306009E52D702E752D0A802912
:101BBB00900001121806FF64786004EFB4581343C9
:101BCB002F01752D1074022529F529E43528F528E8
:101BDB008007E52D7003752D08AB270529E529AA8C
:101BEB00287002052814F91217EDF534C3946140DF
:101BFB000AE534D3947A50035334DF74D02534F58B
:101C0B0034C3940A400CE5349411406D74F92534B7
:101C1B00F534E534D3952D5060432F01853338854A
:101C2B003237853136853035AF2D7E00E4FCFDAB88
:101C3B0033AA32A931A830121845C8ECC8C9EDC96E
:101C4B00CAEECACBEFCBE4FCFDFEEB2534F533EE4D
:101C5B003AF532ED39F531EC38F530AF33AE32AD14
:101C6B0031FCAB38AA37A936A835D312179F5003CE
:101C7B00021BE4432F04021BE4E52F20E003E48066
:101C8B002DE52B452C452A601EAB27E52924FFF9B2
:101C9B00E52834FFFAEBC0E0EAC0E0E9C0E0AB2A8C
:101CAB00AA2BA92C1218B2E52F30E20774FFFFFE06
:101CBB00FDFC22E52FAF33AE32AD31AC3030E1035A
:041CCB000218942245
:1017ED00BB010689828A83E0225002E722BBFE02FA
:0917FD00E32289828A83E493222D
:10180600BB010CE58229F582E5833AF583E0225097
:1018160006E92582F8E622BBFE06E92582F8E222E1
:0D182600E58229F582E5833AF583E49322FB
:10183300BB010689828A83F0225002F722BBFE0194
:02184300F3228E
:10184500E88FF0A4CC8BF0A42CFCE98EF0A42CFC42
:101855008AF0EDA42CFCEA8EF0A4CDA8F08BF0A4C0
:101865002DCC3825F0FDE98FF0A42CCD35F0FCEB1F
:101875008EF0A4FEA9F0EB8FF0A4CFC5F02ECD39E4
:0F188500FEE43CFCEAA42DCE35F0FDE43CFC2251
:0E189400C3E49FFFE49EFEE49DFDE49CFC2265
:1018A200FAE6FB0808E6F925F0F618E6CA3AF62247
:1018B200BB011A89828A83D0F0D0E0F8D0E0F9D057
:1018C200E0FAD0E0FBE8C0E0C0F00219305016E9BF
:1018D200F8D083D082D0E0F9D0E0FAD0E0FBC08229
:1018E200C083021927BBFE16E9F8D083D082D0E06C
:0F18F200F9D0E0FAD0E0FBC082C083021939229E
:10190100D083D082F8E4937012740193700DA3A375
:1019110093F8740193F5828883E473740293686089
:06192100EFA3A3A380DF89
:09192700EBF608EAF608E9F622E5
:09193000EBF0A3EAF0A3E9F022B8
:09193900EBF208EAF208E9F222DF
:00000001FF
